:020000020000FC
:0200000028C016
:02003C0061C1A0
:02004C0070C181
:100050001EC300E10093F2010FEF0DBF04E00EBFDD
:1000600001E00EBD00E00FBD00E809BF00E000BDEB
:1000700001E009B900E00CBF09E100B906E800BDE4
:1000800006E80CBF579A0C9A549A539A0B9AE19926
:10009000FECF00E00FBB0FEF0EBBE09A0DB304B92B
:1000A00000E401BB00E002BB03E007BB01E008BBCA
:1000B0000FEF0ABBB1E0D3E0F2E051D574D558E0C0
:1000C00046E5B1D44091F201D7D47CD597D500E074
:1000D0000093AC0101E00093AA0102E00093A901A2
:1000E00003E00093A50104E00093A30105E0009361
:1000F000A60106E000939C0107E000939A0108E046
:100100000093990109E0009395010AE0009393019F
:100110000BE0009396010CE000938E010DE000933C
:100120008D010EE000938B010FE00093B10100E11F
:100130000093B20101E10093B40102E10093B80120
:1001400003E10093740104E10093720105E100935F
:100150006C0106E100936A0107E10093690108E17F
:100160000093650109E1009363010AE100936601D0
:100170000BE100935C010CE100935A010DE1009347
:1001800059010EE1009355010FE10093530100E284
:100190000093560101E200934E0102E200934D01EB
:1001A00003E200934B0104E20093470105E2009350
:1001B000710106E20093E80107E20093E40108E21E
:1001C0000093E20109E20093D1010AE20093C90120
:1001D0000BE20093C5010CE20093D8010DE20093FD
:1001E000D4010EE20093D2010FE20093CA0100E3B2
:1001F0000093C60101E30093CC0102E30093780170
:1002000003E30093170104E300931B0105E300934C
:100210001D0106E300931E0107E300932E0108E38E
:100220000093360109E300933A010AE300932701A2
:100230000BE300932B010CE300932D010DE30093DE
:1002400035010EE3009339010FE3009333010FEF03
:1002500000933C01009387010093C3010093E101E7
:100260000093F00100930F0177D2179BFECFF89413
:1002700003B1202F007E2F71003229F4203091F538
:100280006BD2AED43BC0003441F429315CF5203050
:1002900049F1E22FC22F5AD131C0003629F4203063
:1002A00009F5C0D19DD42AC0003831F42931D4F4E5
:1002B0002030C1F0EDD122C0003A41F4293194F44C
:1002C000203081F0E22FC22FFDD118C0003C31F464
:1002D000203041F401E00093F30110C0003E11F41E
:1002E000203001F46FD40AEF34D2159BFDCF03B94F
:1002F0000FEF2FD2159BFDCF03B9B7CF7894B5CFB1
:1003000030E03395839B03C03F3FD9F7189530E029
:100310003395E32FC32F60A96F3F31F0603B11F499
:10032000F4D002C0639560AB383191F71895C0984E
:10033000F8940FB70F930091F301003049F02CB1FE
:100340005F9BFECF4CB15F9BFECF5CB1F8D176C016
:100350002CB15C9973C0122F2F71107E203041F0A8
:10036000293134F4103029F0103219F0103409F02A
:1003700065C062E03FEF6A956030C9F13A95303070
:10038000C9F35F9BFBCF4CB15C9958C0473721F153
:1003900030E040FD339541FD339542FD339543FDFB
:1003A000339544FD339545FD339546FD339547FD23
:1003B00033953430F1F54DD04034DCF5042F0C7317
:1003C000043029F0083019F0003009F032C062E042
:1003D0003FEF6A95603011F13A953030C9F35F9B79
:1003E000FBCF5CB15C992AC0573709F101C026C028
:1003F00030E050FD339551FD339552FD339553FD5B
:10040000339554FD339555FD339556FD339557FD82
:100410003395343071F4C22FE22F01C00FC038A9D8
:1004200016FF02C010E03F71312B38AB15D0549845
:1004300016D000A90F3F11F000E000AB54980CB1AA
:100440000BB10F7E0BB90F910FBFC09A549A7894DD
:100450001895A42F4C910895A52F5C9108954737C6
:1004600039F4573729F487E797E715D031D0089545
:10047000479547954795407C003051F0043021F472
:10048000542B852F08D00895542B952F21D00895F3
:10049000542B93D00895E22FC22F18A9312F1F702B
:1004A000307F008D081711F011E0808F103069F057
:1004B000139514FF0AC010E00081081731F0808303
:1004C000988D988343D000E000AB132B18AB0895B0
:1004D000E22FC22F18A9312F1F70307F088D091706
:1004E00011F011E0988F103069F0139514FF0AC0D5
:1004F00010E00881091731F09883808D808326D021
:1005000000E000AB132B18AB08950FEF0083008FB2
:1005100000AB0883088F00E008AB1BD1159BFDCF13
:100520000CEF03B916D1159BFDCF33B900E011D103
:1005300000E0159BFCCF03B90CD1159BFDCF03B98F
:1005400008D1159BFDCF0FEF03B908952931A4F50C
:100550000B9A8081988118A98F3F19F480E090E070
:1005600015C0873799F08F7788320CF409C00FEFE8
:100570000083008F00AB0883088F00E008AB1CC02D
:100580001072103211F08F7701C08068E2D0159B95
:10059000FDCF0CEF03B9DDD0159BFDCF23B9D9D02A
:1005A000159BFDCF83B9D5D0159BFDCF93B9D1D085
:1005B000159BFDCF0FEF03B908954091F601403030
:1005C00031F04091F501541741F40DD00895509346
:1005D000F50141E04093F601089540E04093F501B4
:1005E0004093F60108952931B8F40B9AF2E0E22F16
:1005F00000E000ABAED0159BFDCF0EEF03B9A9D044
:10060000159BFDCF23B9A5D0159BFDCF53B9A1D024
:10061000159BFDCF0FEF03B900E00093F5010093A8
:10062000F6010895E199FECF00E00FBB00EF0EBB8D
:10063000E09A4DB3E199FECF00E00FBB01EF0EBB96
:10064000E09A5DB38091F201E199FECF00E00FBB2B
:1006500003EF0EBBE09A9DB37CD0159BFDCF0DEF51
:1006600003B977D0159BFDCF43B973D0159BFDCF50
:1006700053B96FD0159BFDCF83B96BD0159BFDCFC0
:1006800093B967D0159BFDCF0FEF03B90895189567
:100690003F9300E402BB00E003955D9BFECF2CB9C5
:1006A0003FEF3A950000000000000000000000004D
:1006B000000000003030A9F7003071F700E002BB05
:1006C0003F91089580819881408D588D18A960A927
:1006D00040D0159BFDCF01ED03B93BD0159BFDCF5D
:1006E00083B937D0159BFDCF93B933D0159BFDCF80
:1006F00002ED03B92ED0159BFDCF43B92AD0159B2F
:10070000FDCF53B926D0159BFDCF03ED03B921D002
:10071000159BFDCF13B91DD0159BFDCF63B919D023
:10072000159BFDCF04ED03B904B113D0159BFDCF8C
:1007300003B90FD0159BFDCF0FEF03B90895159B9B
:10074000FECF23B9159BFECF43B9159BFECF53B9FE
:1007500008958299FECF08950F9350D200E0009340
:10076000F3010FEF009301020093020200930302D2
:10077000009304020093050200930602009307020F
:10078000009308020093090200930A0200930B02EF
:1007900000930C0200930D0200930E0200930F02CF
:1007A00000931002009311020093120200931302AF
:1007B000009314020093150200931602009317028F
:1007C00000931802009301030093020300930303B4
:1007D00000930403009305030093060300930703AB
:1007E000009308030093090300930A0300930B038B
:1007F00000930C0300930D0300930E0300930F036B
:10080000009310030093110300931203009313034A
:10081000009314030093150300931603009317032A
:10082000009318030093190200931A0200931B020D
:1008300000931C0200931D0200931E0200931F02EE
:1008400000932002009321020093220200932302CE
:1008500000932402009325020093260200932702AE
:10086000009328020093290200932A0200932B028E
:1008700000932C0200932D0200932E0200932F026E
:10088000009330020093190300931A0300931B0393
:1008900000931C0300931D0300931E0300931F038A
:1008A000009320030093210300932203009323036A
:1008B000009324030093250300932603009327034A
:1008C000009328030093290300932A0300932B032A
:1008D00000932C0300932D0300932E0300932F030A
:1008E0000093300300E00093310200933202009342
:1008F00033020093340200933502009336020093D2
:100900003702009338020093390200933A020093B1
:100910003B0200933C0200933D0200933E02009391
:100920003F02009340020093410200934202009371
:100930004302009344020093450200934602009351
:10094000470200934802009331030093320300935F
:10095000330300933403009335030093360300936D
:100960003703009338030093390300933A0300934D
:100970003B0300933C0300933D0300933E0300932D
:100980003F0300934003009341030093420300930D
:1009900043030093440300934503009346030093ED
:1009A0004703009348030093F5010093F6010F916C
:1009B00008950F9305E80A95F1F70F9108950F93A5
:1009C0005F9301E459EC5A95F1F70A95D9F75F91D5
:1009D0000F9108953F9333E0F2DF3A953030E1F71D
:1009E0003F91089540E435D048E011D043E00FD066
:1009F00043E10DD043E10BD04FE109D04FE107D0E7
:100A000045E105D040E003D040E823D008954F935E
:100A1000407F4BBBD99A18D04F914295407F4BBB3A
:100A2000D99A12D008954F93452F406812D04F9114
:100A30004F93407F4BBBD99A07D04F914295407F4F
:100A40004BBBD99A01D00895DA9AB3DFDA98B1DFB7
:100A500008954F93407F4BBBF7DF4F914295407F06
:100A60004BBBF2DFACDF089541E0F3DFA8DF089570
:100A700042E0EFDFA4DF0895E894542F40E354569A
:100A800010F04395FCCF403311F0689401C040E270
:100A9000BEDF5C5940E35A5010F04395FCCF1EF086
:100AA000403309F440E2B3DF565F40E3450FAFDF68
:100AB0000895E894542F40E3545610F04395FCCF2A
:100AC000403311F0689401C040E2A1DF5C5940E37B
:100AD0005A5010F04395FCCF1EF0403309F440E229
:100AE00096DF565F4EE293DF40E3450F90DF0895B7
:100AF0004FE2E894439580519742E0F7805F984D2C
:100B0000403311F0689401C040E281DF4FE2439529
:100B1000885E9340E0F788519C4F2EF0403311F0EF
:100B2000689401C040E273DF4FE2439584569040E1
:100B3000E0F78C592EF0403311F0689401C040E288
:100B400066DF4FE243958A50E8F7865F1EF0403338
:100B500009F440E25CDF40E3480F59DF089504E008
:100B60002EDF0A950030E1F700E30BBB6DDF27DFD6
:100B70006BDF25DF69DF23DF00E20BBB65DF1FDFF3
:100B800041E267DF4CE165DF42E563DF49E661DFB3
:100B900043E75FDF48E25DDF4CE05BDF41E059DFC8
:100BA00046E057DF089542E532DF43E430DF4DE2AF
:100BB0002EDF4CE42CDF49E62ADF4EE628DF4BE649
:100BC00026DF08954F935F935CE040E22CDF41E421
:100BD0001EDF45E71CDF43E71ADF5F914F91089561
:100BE0004F935F935CE040E21EDF45E410DF49E68F
:100BF0000EDF4EE60CDF5F914F9108954F935F93A8
:100C000050E140E210DF49E402DF4EE600DF49E652
:0C0C1000FEDE44E7FCDE5F914F9108958A
:00000001FF
